:020000000528D1
:080008000900E82404309F0008
:10001000CF3085007F308600F0308700E5248501F1
:1000200086018701882403308700D2249624033078
:100030008700D224962403308700D22496240230ED
:100040008700D22496242830D7240830D7240C30B7
:10005000D7240130D72481244030D7240516962494
:100060000130DF005F08E0000930DE00DE0B3928D8
:100070003F28FF30E00D031C0301D72436285F081A
:10008000FF3A031947285F08DF07DF0A3228051205
:1000900096248030D7240130D724051696242030AA
:1000A000D7245330D7245730D7245230D7242F3079
:1000B000D7245730D7244130D7245430D724543054
:1000C000D7242030D7244D30D7244530D72454307E
:1000D000D7244530D7245230D7242030D7240512D6
:1000E0009624C030D724051696242030D7242030FB
:1000F000D7242030D7242030D7242030D7242030D4
:10010000D7242030D7242030D7242030D7242030C3
:10011000D7242030D7242030D7242030D7242030B3
:10012000D7242030D7242030D7247A247A24EB24F3
:1001300000308D00EE248C130C14EB240C08E52405
:10014000553A0319AA285F30D6000030EC00C830B9
:10015000ED008923EB2401308D00EE248C130C1468
:10016000EB240C08E524D600EB2402308D00EE24AD
:100170008C130C14EB240C08E524EC00EB24033066
:100180008D00EE248C130C14EB240C08E524ED00F8
:10019000071ACD28071ECA28312A2030AB00AC0030
:1001A000AD00AE00AF00B000B100B200B300B400CB
:1001B000B500B600B700B800B900BF00C000C90064
:1001C0002D30D400D500CF00D0000530BC002E303B
:1001D000D3007730C8005030C100C701C601E2012A
:1001E000E601CB23882441309F0096241F151F1958
:1001F000F7281E08E10049309F0096241F151F199B
:10020000FF281E08E4006108CC00AA244C08E10085
:100210006408CC00AA244C08E400640861070318B1
:100220001A291E3C031C1A294708143C031CC82821
:10023000C70AF228C701C60A0030AB000130AC0083
:10024000AD000230AE00AF000330B000B1000430AA
:10025000B200B3000530B400B5000630B600B700F8
:100260000730B800B9001130610203183929203075
:10027000AB002230610203183F292030AC0033303C
:100280006102031845292030AD0044306102031893
:100290004B292030AE00553061020318512920301F
:1002A000AF0066306102031857292030B000773064
:1002B000610203185D292030B10088306102031803
:1002C00063292030B2009930610203186929203077
:1002D000B300AA30610203186F292030B400BB308C
:1002E0006102031875292030B500CC306102031873
:1002F0007B292030B600DD306102031881292030CF
:10030000B700EE306102031887292030B800FE30B4
:10031000610203188D292030B900F12346080F3CF3
:1003200003189529C601E201E60164086602031874
:100330009B296408E600610862020318A32961088A
:10034000E200C601F2286208E1002E245030BF000E
:100350007730C0002030C1004808303A031DC3295F
:100360002030C800BF005030C0007730C1004908BD
:10037000303A031DC3292030C900BF00C0005030EF
:10038000C1007730C8000030A5006208A600003028
:10039000A7006608A80033250030A0002708A100A8
:1003A0002808A2000030A9006430AA0040252308D4
:1003B000CB002408CC000030A5006608A600003061
:1003C000A7006208A80032252708A9002808AA006B
:1003D0000030A000A1004B08A2004C08A300872514
:1003E0002208A5002308A6000030A7000530A800B9
:1003F00033250030A000A100A9002708A20028088A
:10040000A3000A30AA0087252208E3002308E5009C
:10041000F1246908003A031D112A6808043C0318F6
:10042000272ABC0B172A0730BC000130BA063A1C39
:10043000202A4830D4004930D3004730D5002F2A35
:100440002030D4002030D3002030D5002F2A680877
:10045000303ED4006708303ED5002E30D300CB2389
:10046000F228AB01AC01AD01AE01AF012030B0000C
:10047000B10041309F006C08E3006D08E500F124F5
:100480006708303EBD006808303EDB006908303E3A
:10049000BE006A08303EEE006E08303A031D582A4E
:1004A0002030EE003E08303A031D582A2030BE00AE
:1004B000051296240230D724051696244330D724FB
:1004C0004130D7244C30D7244930D7244230D72468
:1004D0005230D7244130D7245A30D7244930D7243A
:1004E0004F30D7244E30D7244530D7242030D7245E
:1004F0002030D7243008D7243108D7240512962479
:10050000C030D724051696246930D7246E30D724FE
:100510007030D7247530D7247430D7242030D724B6
:100520007730D7246130D7247430D7247430D7245F
:100530002030D7242B18A82A2B146E08D7243E0865
:10054000D7245B08D7242E30D7243D08D724B82AD7
:100550002B102030D7242030D7242030D72420302F
:10056000D7242030D724C830AC00AC0BC32A3B2A98
:10057000AC0BBB2A3B2A8F24871ADE018F24071B72
:10058000DF018F24B82A8F24871AE32ADE0A093074
:10059000AD005E08083C0318AD01AD0A00306C06E2
:1005A0000319D82A2D08ED020318B82AEC03B82A3B
:1005B0002D08ED026D08313C031CB82A0330EC0015
:1005C000E830ED00B82A8F24071B022BDF0A093020
:1005D000AD005F08083C0318AD01AD0A03306C069E
:1005E0000319F82A2D08ED07031CB82AEC0AB82ACB
:1005F0002D08ED07E9306D02031CB82AEC013230FA
:10060000ED00B82A8F24071E072B1824B52A071ED1
:10061000072BAD014F303006031D9728FF30E10056
:100620002E24C830AC00051296240130D7240516BC
:1006300096244630D7247330D7246330D7246130D2
:10064000D7246C30D7246130D7242030D7246D30A4
:10065000D7246130D7247830D7242030D7244808D5
:10066000D7244908D7244F08D7242E30D724500840
:10067000D72405129624C030D724051696246D3051
:10068000D7246530D7246D30D7246F30D72472300B
:10069000D7246930D7247A30D7247A30D7246F30E2
:1006A000D7243F30D7242030D7245330AD18203002
:1006B000D7244930AD182030D7242030D7244E30ED
:1006C0002D182030D7244F302D182030D724AC0BD4
:1006D000732B2D1D6F2B2D100230AD06112BAD107D
:1006E0000130AD06112B8F24871A7A2B871E762BAB
:1006F0000430AD068F24071B812B071F7D2B043090
:10070000AD068F24071A672B071E842B2D1989230A
:100710009728EB2455308C0000308D00EE248C138C
:100720000C1555308D00AA308D008C140C118824C6
:10073000E524E5245608EB248C0001308D00EE24DE
:100740008C130C1555308D00AA308D008C140C11B3
:100750008824E5246C08EB248C0002308D00EE2404
:100760008C130C1555308D00AA308D008C140C1193
:100770008824E5246D08EB248C0003308D00EE24E2
:100780008C130C1555308D00AA308D008C140C1173
:100790008824E5240800051296240230D724051683
:1007A00096245330D7245730D7245230D7242030C2
:1007B000D7245408D7245308D7245508D7242030E9
:1007C000D7243F08D7244008D7244108D724480815
:1007D000D7244908D7244F08D7242E30D7245008CF
:1007E000D72405129624C030D7240516962400304D
:1007F000D7242B08D7242C08D7242D08D7242E083B
:10080000D7242F08D7243008D7243108D72432081A
:10081000D7243308D7243408D7243508D7243608FA
:10082000D7243708D7243808D7243908D724080014
:100830001F151F19192C1E08193C031808001E0843
:10084000CC00AA244C08D6002E0203180800560833
:10085000AE004F30B0004B30B10008000030A000B7
:10086000A100A9005608A200AA0040252308D10033
:100870002408D2000030A000A100A9006108A20055
:10088000AA0040252308A1002408A2000030A900E6
:100890006430AA0040252208A0002308A1002408F3
:1008A000A2006C08A9006D08AA0040252108A0003C
:1008B0002208A1002308A2002408A3005108A900CF
:1008C0005208AA0087250030A9006430AA008725B5
:1008D0002208E3002308E500F1246A08303EC8003E
:1008E0006908303EC9006808303ECF006708303ED6
:1008F000D00008000730C2006430C300FF30C400DD
:10090000A32C0230C2003230C300FF30C400A32C3D
:100910000130C2001430C300FF30C400A32C0130EA
:10092000C2000130C300C830C400A32C0130C20093
:100930000730C3009330C400A32C0130C400013041
:10094000C2000130C300C40BA32CC30BA32CC20BE9
:10095000A32C0800F1304C02031CB12CFF30CC005A
:1009600008007B304C02031CB72C0E30D02C2A30F0
:100970004C02031CBD2C0C30D02C0D304C02031C3F
:10098000C32C0A30D02C06304C02031CC92C083072
:10099000D02C03304C02031CCF2C0630D02C00305E
:1009A000CC07080085169D2485129D240800C500EB
:1009B000450E870085169D2485129D2445088700D5
:1009C00085169D2485129D240800031383120800B8
:1009D00003138316080003178312080003178316F6
:1009E0000800E701E801E901EA01EB016308003AC8
:1009F00003190E2D0025E30BFE2C0E2D0025FB2CDC
:100A0000242524251E251E251E251E251E251825C8
:100A10001825182518251825182508000030650602
:100A2000031908001825E50B162D08001825132DAD
:100A3000E70A67080A3A031D0800E701E80A6808A0
:100A40000A3A031D0800E801E90A69080A3A031D89
:100A50000800E901EA0A6A080A3A031D0800EA01E7
:100A6000EB0A08003A252608A8070318A70A250854
:100A7000A7070034A609A60A0319A503A50900348F
:100A8000A301A4012008D8002108D9002208DA0017
:100A90000830BB00AA0C03185B2DBB0B4A2DBB0012
:100AA000A90C0318592DBB0B502DA001A101A201C7
:100AB000003403107F2D03106A2DAA0C031C6A2D2D
:100AC0005A08A20759080318590FA1075808031814
:100AD000580FA007A00CA10CA20CA30CBB0B5D2D02
:100AE0000830BB00A90C031C7F2D5A08A207590827
:100AF0000318590FA10758080318580FA007A00C96
:100B0000A10CA20CA30CA40CBB0B722D0800D101EC
:100B1000D201D701200DD20D2A08D2022908031CC8
:100B2000290FD1020301031C0130D702A00D0730A9
:100B3000BB00200DD20DD10DD70D2A08201CAA2DE7
:100B4000D2022908031C290FD1020301031C013022
:100B5000D702B32DD20729080318290FD1070301A3
:100B600003180130D707A00DBB0B992D210DD20D15
:100B7000D10DD70D2A08201CC72DD2022908031C2D
:100B8000290FD1020301031C0130D702D02DD20757
:100B900029080318290FD107030103180130D707CB
:100BA000A10D0730BB00210DD20DD10DD70D2A08A4
:100BB000211CE42DD2022908031C290FD1020301B4
:100BC000031C0130D702ED2DD20729080318290F85
:100BD000D107030103180130D707A10DBB0BD32D9B
:100BE000220DD20DD10DD70D2A08211C012ED202C3
:100BF0002908031C290FD1020301031C0130D7026D
:100C00000A2ED20729080318290FD1070301031858
:100C10000130D707A20D0730BB00220DD20DD10D38
:100C2000D70D2A08221C1E2ED2022908031C290FC8
:100C3000D1020301031C0130D702272ED207290855
:100C40000318290FD107030103180130D707A20D9C
:100C5000BB0B0D2E230DD20DD10DD70D2A08221C52
:100C60003B2ED2022908031C290FD1020301031CC9
:100C70000130D702442ED20729080318290FD107C3
:100C8000030103180130D707A30D0730BB00230D64
:100C9000D20DD10DD70D2A08231C582ED2022908B7
:100CA000031C290FD1020301031C0130D702612E5E
:100CB000D20729080318290FD107030103180130AF
:100CC000D707A30DBB0B472E23186C2E2A08D2077B
:0A0CD00029080318290FD1070800B6
:02400E00313F40
:00000001FF
